:100000000000001C22021A2A2A1C00000000000026
:10001000000000081422223E2222000000000000FE
:100020000000003C12121C12123C000000000000F4
:100030000000001C22202020221C000000000000E4
:100040000000003C12121212123C000000000000DE
:100050000000003E20203820203E0000000000006C
:100060000000003E2020382020200000000000007A
:100070000000001E20202622221E0000000000009A
:100080000000002222223E22222200000000000066
:100090000000001C08080808081C00000000000000
:1000A0000000000202020222221C000000000000E8
:1000B0000000002224283028242200000000000034
:1000C0000000002020202020203E00000000000032
:1000D00000000022362A2A2222220000000000000E
:1000E00000000022322A2622222200000000000006
:1000F0000000003E22222222223E000000000000DA
:100100000000003C22223C202020000000000000D3
:100110000000001C2222222A241A000000000000F5
:100120000000003C22223C282422000000000000A5
:100130000000001C22100804221C00000000000027
:100140000000003E08080808080800000000000041
:100150000000002222222222221C000000000000B7
:1001600000000022222214140808000000000000F1
:100170000000002222222A2A36220000000000006D
:1001800000000022221408142222000000000000B7
:1001900000000022221408080808000000000000E7
:1001A0000000003E02040810203E00000000000095
:1001B000000000382020202020380000000000002F
:1001C00000000020201008040202000000000000CF
:1001D0000000000E02020202020E000000000000F9
:1001E000000000081C2A08080808000000000000A1
:1001F0000000000008103E10080000000000000091
:1002000000000000000000000000000000000000EE
:1002100000000008080808080008000000000000AE
:100220000000001414140000000000000000000092
:100230000000001414360036141400000000000002
:10024000000000081E201C023C0800000000000006
:1002500000000032320408102626000000000000D2
:10026000000000102828102A241A000000000000B6
:100270000000001818180000000000000000000036
:1002800000000008102020201008000000000000DE
:100290000000000804020202040800000000000040
:1002A00000000000081C3E1C0800000000000000C8
:1002B0000000000008083E080800000000000000E0
:1002C000000000000000303010200000000000009E
:1002D0000000000000003E000000000000000000E0
:1002E00000000000000000003030000000000000AE
:1002F000000000020204081020200000000000009E
:100300000000001824242424241800000000000009
:100310000000000818080808081C00000000000081
:100320000000001C22021C20203E000000000000F3
:100330000000001C22020402221C00000000000039
:10034000000000040C143E0404040000000000003F
:100350000000003E203C0202221C000000000000C1
:100360000000001C20203C22221C00000000000095
:100370000000003E020408102020000000000000E1
:100380000000001C22221C22221C00000000000091
:100390000000001C22221E02021C000000000000BF
:1003A00000000000181800181800000000000000ED
:1003B00000000018180018180810000000000000C5
:1003C00000000004081020100804000000000000D5
:1003D00000000000003E003E0000000000000000A1
:1003E00000000010080402040810000000000000D3
:1003F00000000018240408080008000000000000A5
:00000001FF
